:020000040000FA
:040000001FD00ED02F
:0400080004EF04F00D
:040018000CEF04F0F5
:10002000A66E05A01200550EA76EAA0EA76EA68298
:100030000000A6B2FED712000A26D8B00B2A120082
:10004000A66AA968AA68A680A83C00EF04F0066A20
:100050001C0E056E0F019394000E006F080E016FC9
:10006000E81E056F000E026F070E036FFF0E186F7C
:10007000EB0E196FFF0E1A6FF80E1B6F030E706EEA
:100080009E0E716E030E726E200E736E6F6A939EDB
:10009000939C819E818C0400609E60AEFED70FEE23
:1000A00066F065500F0B096EF46EF5E064B02BD06E
:1000B00010EE01F0EECFE6FFF42EFCD70650EBE099
:1000C000010AD8A407D0A968AA68A86A040EA8DF04
:1000D000819CFF000650020A05E10B6A0A6A0C9037
:1000E0000C6AD9D70650030A0AE107500A2606E12E
:1000F00008500B2203E10CB001D073D076D006502B
:10010000040AC9E176D00350F86EF00BF36E02508A
:10011000F76EAA6E0150F66EA96E05A605D00950BD
:100120000126E86A02220322300EF36001D008D0D3
:10013000F350300A01E12AD0F350F00AACE132D09A
:1001400005A405D0F6503F0B02E1940E69DF05B21D
:10015000A2D7F650070B9FE1080EF46EEE50F56E35
:100160006BDF0D00F42EFAD7080EF46E0A00ED5086
:10017000F42EFCD7840E54DF080EF46E0900F550FF
:10018000EE18D8A40C80F42EF9D785D7EF50F56E71
:1001900053DF0C00C40E44DF0900F550EE18F42EB6
:1001A000F5D779D7EF50A86E47DF040E39DFA66A7E
:1001B000A680A850EE18D8A40C80A94AAA2AF42E2A
:1001C000F1D769D740B7FED7800E416F080E426F56
:1001D000000E436F040E446F448164A04491408735
:1001E0005AD7010E466F456FEDD7466B010E456F2E
:0C01F000E9D7020E466F010E456FE4D700
:0401FC0012EE00F00F
:10020000800E006EA50EE66E002EFDD712EE00F0F9
:1002100022EE00F0F86A519C1CEC04F0DEEC06F0D3
:04022000FBD71200F6
:080800000000FEEF00F0120001
:0808080007ED04F012000600E8
:06081000D5EF04F0120018
:020816000000E0
:0608180020EF04F01200C5
:06082A0000EE00F00D0ECF
:08083000EE6AEA62FDD7120036
:020838001200AC
:10084000D8CFE4FFE0CFE4FFE46EDACFE4FFE2CFFD
:10085000DAFFE652A4A004D00F0140871588A390C8
:10086000A4AA02D000000000A46AE552E5CFDAFF96
:10087000E550E5CFE0FFE5CFD8FF10001494E0C2CB
:10088000E9FFE1C2EAFF060EEB505C0A56E0190AE6
:1008900051E0040A43E04B0A3EE0020A39E0010A53
:1008A00037E0890A32E0200A30E0600A2EE0200AB0
:1008B0002CE0C20A27E0030A22E0650A1DE0040AD0
:1008C00018E0C40A13E0260A11E0200A0FE0010A2A
:1008D0000DE0A00A08E0640A03E0270A01E054D012
:1008E00030EC0AF052D062EC10F04FD0BAEC16F0B7
:1008F0004CD010EC09F049D0FAEC09F046D0CEEC1F
:100900000FF043D021EC0FF040D078EC10F03DD048
:1009100059EC16F03AD050EC11F037D0630E426E1D
:10092000436A446A040E456E040EE66EE8EC1AF063
:10093000E5522BD083EC11F028D0E0C2E9FFE1C2F0
:10094000EAFF070EEB504C6E4D6AE0C2E9FFE1C2D0
:10095000EAFF080EEB50080F4CC04AF04DC04BF0B8
:1009600005E0D8904A364B36E804FBE1720E4A188F
:1009700001E14B5008E1E668FF0EE66ED5EC19F098
:10098000E552E552FF0001D000D014B40DD00000B4
:10099000E0C2E9FFE1C2EAFFEF6A15A804D01598AA
:1009A000A380E1EC1AF000D01200DACFE4FFE2CF2E
:1009B000DAFFE9CFE4FFEACFE4FFE652F2941A50FF
:1009C000D66E81AA15D015A008D015A203D08294A6
:1009D000828202D08292828402D08292829415A472
:1009E00006D01550080B02E0828601D0829614D002
:1009F00015A408D015A603D08294828202D08292D8
:100A0000828402D08292829415A006D01550020BE7
:100A100002E0828601D0829615A002D0818C01D09E
:100A2000819C15A402D0818E01D0819E010E0F5EA3
:100A3000000E105A115A0F501010111007E1650ED8
:100A40000F6E0D0E106E010E116E158A00500C0AFD
:100A500001E199D0070A01E193D0010A01E18CD0AC
:100A6000030A01E187D0010A01E180D00F0A74E096
:100A7000010A6EE0030A55E0010A50E0070A4AE065
:100A8000010A10E0030A0DE0010A01E07CD01572B2
:100A9000800E0214800802E1010E01D0040E006EE7
:100AA00076D01572006A0250E824026E09060950D9
:100AB00001E06DD00D2A0D50EA6A1E0FE96E000E9E
:100AC000EA22EF50026E080E096E040604501FE180
:100AD0002406245006E01350100B07E11250080BB7
:100AE00004E0060E006E128011D0080E006E0D6A32
:100AF0000D50EA6A1E0FE96E000EEA22EF50026EF8
:100B00000850036E0B50046E080E096E02D00C0ED6
:100B1000006E3DD01572020E006E39D0030E006ECD
:100B200036D01572060E006E12B011D0080E006E8F
:100B30000D6A0D50EA6A1E0FE96E000EEA22EF50B0
:100B4000026E0850036E0B50046E080E096E1FD023
:100B50001572050E006E1BD015720306035003E1DB
:100B60000C0E006E02D0080E006E11D01572070E2A
:100B7000006E0DD0006A0BD01572090E006E07D002
:100B80000A0E006E04D015720B0E006E00D00150DC
:100B90000C0A01E193D0070A01E18DD0010A01E1BD
:100BA00086D0030A01E181D0010A01E17AD00F0A5F
:100BB0006EE0010A68E0030A4FE0010A4AE0070A12
:100BC00044E0010A10E0030A0DE0010A01E076D0DA
:100BD0001576800E0514800802E1010E01D0040E86
:100BE000016E70D01576016A0550E824056E0A067C
:100BF0000A5001E067D00E2A0E50EA6A250FE96E0E
:100C0000000EEA22EF50056E080E0A6E0706075026
:100C100019E12B062B5004E1060E016E138011D052
:100C2000080E016E0E6A0E50EA6A250FE96E000E7C
:100C3000EA22EF50056E0E0E066E0C50076E080E7F
:100C40000A6E02D00C0E016E3DD01576020E016EBA
:100C500039D0030E016E36D01576060E016E13B034
:100C600011D0080E016E0E6A0E50EA6A250FE96E69
:100C7000000EEA22EF50056E0E0E066E0C50076E47
:100C8000080E0A6E1FD01576050E016E1BD0157664
:100C90000606065003E10C0E016E02D0080E016E2E
:100CA00011D01576070E016E0DD0016A0BD01576A6
:100CB000090E016E07D00A0E016E04D015760B0ED8
:100CC000016E00D01850040A6EE0070A69E0010ABC
:100CD0000CE0030A06E0010A01E068D0010E186E7C
:100CE00065D0020E186EC28261D0C2B258D0C45014
:100CF0004E6E4EC04FF04E6AC35000014E10606FF2
:100D00004FC061F06251645D646F63516559656FF6
:100D100064516025646F65516121656F64C062F044
:100D200065C063F0D89063336233D8906333623325
:100D3000010EC26E030E186E165023E112AA0BD0DC
:100D4000050E19244E6E4F6A4E50625D4F50635926
:100D500001E3128615D0000E605D030E61590DE2AD
:100D600012AC0AD017504E6E4F6A4E50625D4F5013
:100D7000635902E3020E166E03D015901288129C7E
:100D80000ED0160616500BE117504E6E4F6A4E509D
:100D9000625D4F50635903E315901288129C06D090
:100DA000040E186E03D0010E186E00D0E552E5CF88
:100DB000EAFFE5CFE9FFE5CFDAFF1100D9CFE6FF83
:100DC000E1CFD9FFE6525CD81584DF6A050EDF5CFF
:100DD00009E2070E426E010EE66EE8EC1AF0E552EB
:100DE000DF2AF4D712B812981350020B03E1135004
:100DF000040B05E01250010B02E044EC17F013A0C5
:100E000002D0F8EC08F092EC1AF0000902E13EEC96
:100E100004F015AA2FD0DF6A200EDF5C2AE2DF5033
:100E2000080DF3CFE9FFF4CFEAFF000EE926010E2B
:100E3000EA22EF50800B1BE0DF50080DF3CFE9FFF3
:100E4000F4CFEAFF000EE926010EEA22070EE9269A
:100E5000000EEA22EF060BE1DF50080DF3CFE9FFA9
:100E6000F4CFEAFF000EE926010EEA22EF9EDF2A08
:100E7000D3D7159AB7D7E552E552E7CFD9FF12007D
:100E8000D9CFE6FFE1CFD9FFE652F26AA66A159004
:100E90001594826A816A806AF00E946E3F0E936E9A
:100EA000FB0E926E828089EC19F0A56AA26A9F6A95
:100EB000210EA36EA06A9D6AF06AF16AF26AA46AC2
:100EC000A16A9E6AD08E166A060E006E016E126AC4
:100ED000136A13801280DF6A200EDF5C66E2DF5047
:100EE000080DF3CFE9FFF4CFEAFF000EE926010E6B
:100EF000EA22EF6ADF50080DF3CFE9FFF4CFEAFFF3
:100F0000000EE926010EEA22EE52EE6AED6ADF508B
:100F1000080DF3CFE9FFF4CFEAFF000EE926010E3A
:100F2000EA22030EE926000EEA22800EEF6EDF5061
:100F3000080DF3CFE9FFF4CFEAFF000EE926010E1A
:100F4000EA22040EE926000EEA22EF6ADF50080DBD
:100F5000F3CFE9FFF4CFEAFF000EE926010EEA2203
:100F6000050EE926000EEA22EF6ADF50080DF3CFE6
:100F7000E9FFF4CFEAFF000EE926010EEA22060E91
:100F8000E926000EEA22EF6ADF50080DF3CFE9FFF1
:100F9000F4CFEAFF000EE926010EEA22070EE92649
:100FA000000EEA22EF6ADF2A97D72C6A2D6ADF6AE1
:100FB000100EDF5C01E378D0DF50080DF3CFE9FFBE
:100FC000F4CFEAFF600EE926020EEA22EF6ADF5054
:100FD000080DF3CFE9FFF4CFEAFF600EE926020E19
:100FE000EA22EE52EF6ADF50080DF3CFE9FFF4CFAB
:100FF000EAFF600EE926020EEA22EE52010EE92611
:10100000000EEA22EF6ADF50080DF3CFE9FFF4CFBC
:10101000EAFF600EE926020EEA22EE52020EE926EF
:10102000000EEA22EF6ADF50080DF3CFE9FFF4CF9C
:10103000EAFF600EE926020EEA22EE52030EE926CE
:10104000000EEA22EF6ADF50080DF3CFE9FFF4CF7C
:10105000EAFF600EE926020EEA22EE52040EE926AD
:10106000000EEA22EF6ADF50080DF3CFE9FFF4CF5C
:10107000EAFF600EE926020EEA22EE52050EE9268C
:10108000000EEA22EF6ADF50080DF3CFE9FFF4CF3C
:10109000EAFF600EE926020EEA22070EE926000E9C
:1010A000EA22EF6ADF2A84D72E6A2F6A92EC1AF0BE
:1010B000000906E1E0C2E9FFE1C2EAFFEF6AF6D704
:1010C000146A34EC16F0E66AC5EC19F0E5525D08D6
:1010D00005E0146A600E176E41EC16F0860EC06EC5
:1010E0000E0EC16E010EC26E186A196A650E0F6E81
:1010F0000D0E106E010E116E400ED56ED66AD76AB7
:10110000F28AD58EF184970E1A6E14AA02D0A30E1D
:101110001A6E386A0001626B636B0001646B656B69
:101120003C6ABE0E3D6EE00E3E6E0F017E0E416FBC
:10113000E00E426F010E456F020E466FF28EF28C8A
:10114000E552E552E7CFD9FF1200D9CFE6FFE1CF54
:10115000D9FFE652400EDF6EFE0EDB507F0803E241
:10116000200EDF10DF6EFE0EDB507F0B010803E167
:10117000010EDF1011D0FE0EDB507F0BE840E8407F
:10118000E8401F0BDF10DF6EFE0EDBA403D0100E55
:10119000DF10DF6EDF5000D0E552E552E7CFD9FF18
:1011A0001200D9CFE6FFE1CFD9FFE652400EDF6E45
:1011B000FE0EDB504A6E4B6A4A50800B03E0200E55
:1011C000DF10DF6EFE0EDB507F0B010803E1010E26
:1011D000DF1009D0FE0EDB507F0BE840E840E8400E
:1011E0001F0BDF1000D0E552E552E7CFD9FF120008
:1011F000305013E12F50080DF3CFE9FFF4CFEAFF91
:10120000600EE926020EEA22EF50800B03E014EC98
:1012100014F002D098EC14F002D02AEC16F0120070
:10122000D9CFE6FFE1CFD9FF040EE126DE52010E51
:10123000DD6EE0C2E9FFE1C2EAFF070EEB504C6E43
:101240004CC04DF04C6AE0C2E9FFE1C2EAFF080E73
:10125000EB5000014C104A6E4DC04BF0020E4AC0DC
:10126000DBFF030E4BC0DBFFD950020FE96EDACF74
:10127000EAFFEE50ED1001E1B3D0DF6A200EDF5C33
:101280002EE2DF50080DF3CFE9FFF4CFEAFF000EA6
:10129000E926010EEA22EF50800B04E1010EDB6A21
:1012A0001ED01BD0DF50080DF3CFE9FFF4CFEAFFCB
:1012B000000EE926010EEA22EE52EECF4AF0EFCF01
:1012C0004BF0020EDB504A1803E1030EDB504B18C3
:1012D00004E1DE52020EDD6E02D0DF2ACFD7010E0E
:1012E000DB5066E1DF50080DF3CFE9FFF4CFEAFFF2
:1012F000000EE926010EEA22EE52020EDBCFEEFFCF
:10130000030EDBCFEDFFDF50080DF3CFE9FFF4CF85
:10131000EAFF000EE926010EEA22EE52EE52EF50ED
:10132000800B01E0010E4A6EDF50080DF3CFE9FF9C
:10133000F4CFEAFF000EE926010EEA22EE52EE5249
:101340004A50010BF36EF346F346F346F346F34679
:10135000F346BF0EEF14F310EF6EDF50080DF3CF1E
:10136000E9FFF4CFEAFF000EE926010EEA22EF8E34
:10137000E10E426EDF50436EE0C2E9FFE1C2EAFFD8
:10138000070EEB50446EE0C2E9FFE1C2EAFF080E2F
:10139000EB50456E0BC146F00CC147F00DC148F053
:1013A0000EC149F0080EE66EE8EC1AF0E55218D0CE
:1013B000630E426EE0C2E9FFE1C2EAFF070EEB50A6
:1013C000436EE0C2E9FFE1C2EAFF080EEB50446E53
:1013D000010EDB50456E040EE66EE8EC1AF0E552A5
:1013E000040EE15C02E2E16AE552E16EE552E7CF0C
:1013F000D9FF1200E0C2E9FFE1C2EAFF070EEB509D
:10140000080DF3CFE9FFF4CFEAFF000EE926010E45
:10141000EA22EF50800B23E0E0C2E9FFE1C2EAFFDD
:10142000080EEB50030B4A6EE0C2E9FFE1C2EAFF8F
:10143000070EEB50080DF3CFE9FFF4CFEAFF000EE3
:10144000E926010EEA224A50030BF36EF346F346F7
:10145000F346F346F3469F0EEF14F310EF6E1200BF
:10146000D9CFE6FFE1CFD9FF040EE126DF6A2E5087
:10147000080DF3CF4AF0F4CF4BF0600E4A26020E6F
:101480004B22020E4AC0DBFF030E4BC0DBFFE0C263
:10149000E9FFE1C2EAFF070EEB50080DF3CFE9FFC9
:1014A000F4CFEAFF000EE926010EEA22EF50800B8E
:1014B00002E117EF0FF0E0C2E9FFE1C2EAFF070E19
:1014C000EB50080DF3CFE9FFF4CFEAFF000EE92659
:1014D000010EEA22070EE926000EEA22050EEF6E43
:1014E000E0C2E9FFE1C2EAFF060EEB50470821E146
:1014F000E0C2E9FFE1C2EAFF080EEB50E76E010E21
:10150000E7CFDBFFE0C2E9FFE1C2EAFF070EEB50E5
:10151000080DF3CFE9FFF4CFEAFF000EE926010E34
:10152000EA22030EE926000EEA22010EDBCFEFFFCE
:1015300067D0E0C2E9FFE1C2EAFF080EEB50030A00
:1015400041E0010A21E0030A01E05AD0E0C2E9FFCC
:10155000E1C2EAFF090EEB50E66EE0C2E9FFE1C22C
:10156000EAFF070EEB50080DF3CFE9FFF4CFEAFFD7
:10157000000EE926010EEA22040EE926000EEA22F8
:10158000E552E750EF6E3CD0E0C2E9FFE1C2EAFF6E
:10159000090EEB50E66EE0C2E9FFE1C2EAFF070E7A
:1015A000EB50080DF3CFE9FFF4CFEAFF000EE92678
:1015B000010EEA22050EE926000EEA22E552E75066
:1015C000EF6E1ED0E0C2E9FFE1C2EAFF090EEB5068
:1015D000E66EE0C2E9FFE1C2EAFF070EEB50080D3C
:1015E000F3CFE9FFF4CFEAFF000EE926010EEA226D
:1015F000060EE926000EEA22E552E750EF6E00D013
:10160000020EDBCFE9FF030EDBCFEAFFEF50800BCA
:1016100002E015EF0FF0020EDBCFE9FF030EDBCF88
:10162000EAFFEE52050EE926000EEA22EF6AE0C25A
:10163000E9FFE1C2EAFF070EEB50080DF3CFE9FF27
:10164000F4CFEAFF000EE926010EEA22EE52EE5236
:10165000EF50800B01E1A1D0E0C2E9FFE1C2EAFF57
:10166000070EEB50080DF3CFE9FFF4CFEAFF000EB1
:10167000E926010EEA22EE52EE52EF50E66E020E1D
:10168000DBCFE9FF030EDBCFEAFFEE52E9CF4AF0F2
:10169000EACF4BF0DF500F014A24E96E000E4B20D9
:1016A000EA6EE552E750EF6E020EDBCFE9FF030E64
:1016B000DBCFEAFFEE52E9CF4AF0EACF4BF0DF5042
:1016C000DF2A4A24E96E000E4B20EA6EEF50E66EE8
:1016D000020EDBCFE9FF030EDBCFEAFFEE52050E71
:1016E000E926000EEA22E552E750EF6EE0C2E9FF7C
:1016F000E1C2EAFF070EEB50080DF3CFE9FFF4CF8C
:10170000EAFF000EE926010EEA22EE52EF50E66EE5
:10171000020EDBCFE9FF030EDBCFEAFFEE52E9CF8B
:101720004AF0EACF4BF0DF504A24E96E000E4B201E
:10173000EA6EE552E750EF6E020EDBCFE9FF030ED3
:10174000DBCFEAFFEE52E9CF4BF0EACF4CF0DF50AF
:10175000DF2A4B24E96E000E4C20EA6EEFCF4AF0F0
:10176000020EDBCFE9FF030EDBCFEAFFEE52050EE0
:10177000E926000EEA22EF504A18E66E020EDBCF91
:10178000E9FF030EDBCFEAFFEE52050EE926000E5D
:10179000EA22E552E750EF6E49D0E0C2E9FFE1C22C
:1017A000EAFF070EEB50080DF3CFE9FFF4CFEAFF95
:1017B000000EE926010EEA22EE52EF50E66E020E0E
:1017C000DBCFE9FF030EDBCFEAFFEE52E9CF4AF0B1
:1017D000EACF4BF0DF500F014A24E96E000E4B2098
:1017E000EA6EE552E750EF6E020EDBCFE9FF030E23
:1017F000DBCFEAFFEE52E9CF4AF0EACF4BF0DF5001
:10180000DF2A4A24E96E000E4B20EA6EEF50E66EA6
:10181000020EDBCFE9FF030EDBCFEAFFEE52050E2F
:10182000E926000EEA22E552E750EF6EE0C2E9FF3A
:10183000E1C2EAFF060EEB50470801E054D1E0C2D6
:10184000E9FFE1C2EAFF070EEB50080DF3CFE9FF15
:10185000F4CFEAFF000EE926010EEA22EF50600BFA
:10186000E842E842E842E842E842010A01E1AED03B
:10187000020A5DE0010A5BE0020A01E0F7D0020E15
:10188000DBCFE9FF030EDBCFEAFFEE52E9CF4AF0F0
:10189000EACF4BF0DF504A24E96E000E4B20EA6E8F
:1018A0003F0EEF6E020EDBCFE9FF030EDBCFEAFF48
:1018B000EE52E9CF4BF0EACF4CF0DF50DF2A4B2459
:1018C000E96E000E4C20EA6EEFCF4AF0020EDBCF3D
:1018D000E9FF030EDBCFEAFFEE52050EE926000E0C
:1018E000EA22EF504A18E66E020EDBCFE9FF030E44
:1018F000DBCFEAFFEE52050EE926000EEA22E552A2
:10190000E750EF6E020EDBCFE9FF030EDBCFEAFFFD
:10191000EE52E9CF4AF0EACF4BF0DF504A24E96EAD
:10192000000E4B20EA6E010EDBCFEFFF9FD0010EC1
:10193000DBCFE6FF0ADCE552E76E010EE7CFDBFF07
:10194000020EDBCFE9FF030EDBCFEAFFEE52E9CF59
:101950004AF0EACF4BF0DF500F014A24E96E000E47
:101960004B20EA6E010EDBCFEFFF020EDBCFE9FF6B
:10197000030EDBCFEAFFEE52E9CF4BF0EACF4CF09B
:10198000DF50DF2A4B24E96E000E4C20EA6EEFCFC9
:101990004AF0020EDBCFE9FF030EDBCFEAFFEE5287
:1019A000050EE926000EEA22EF504A18E66E020EF6
:1019B000DBCFE9FF030EDBCFEAFFEE52050EE9268F
:1019C000000EEA22E552E750EF6E50D0010EDBCF59
:1019D000E6FFD1EC08F0E552E76E010EE7CFDBFF42
:1019E000020EDBCFE9FF030EDBCFEAFFEE52E9CFB9
:1019F0004AF0EACF4BF0DF500F014A24E96E000EA7
:101A00004B20EA6E010EDBCFEFFF020EDBCFE9FFCA
:101A1000030EDBCFEAFFEE52E9CF4BF0EACF4CF0FA
:101A2000DF50DF2A4B24E96E000E4C20EA6EEFCF28
:101A30004AF0020EDBCFE9FF030EDBCFEAFFEE52E6
:101A4000050EE926000EEA22EF504A18E66E020E55
:101A5000DBCFE9FF030EDBCFEAFFEE52050EE926EE
:101A6000000EEA22E552E750EF6E00D0020EDBCF07
:101A7000E9FF030EDBCFEAFFEE52E9CF4BF0EACFEE
:101A80004CF0DF50DF2A4B24E96E000E4C20EA6E4A
:101A9000EFCF4AF0020EDBCFE9FF030EDBCFEAFF08
:101AA000EE52050EE926000EEA22EF504A18E66EC5
:101AB000020EDBCFE9FF030EDBCFEAFFEE52050E8D
:101AC000E926000EEA22E552E750EF6E020EDBCF68
:101AD000E9FF030EDBCFEAFF070EE926000EEA223C
:101AE000010EEF6E66D1E0C2E9FFE1C2EAFF080E27
:101AF000EB50050A01E1C2D0010A61E0070A41E0AA
:101B0000010A21E0030A01E018D1E0C2E9FFE1C2C5
:101B1000EAFF090EEB501F0B8009E66E020EDBCFC9
:101B2000E9FF030EDBCFEAFFEE52E9CF4AF0EACF3E
:101B30004BF0DF504A24E96E000E4B20EA6EE5526E
:101B4000E750EF6EFAD0E0C2E9FFE1C2EAFF090E0A
:101B5000EB500F0BB009E66E020EDBCFE9FF030E70
:101B6000DBCFEAFFEE52E9CF4AF0EACF4BF0DF508D
:101B70004A24E96E000E4B20EA6EE552E750EF6E04
:101B8000DCD0E0C2E9FFE1C2EAFF090EEB500F0B27
:101B9000A009E66E020EDBCFE9FF030EDBCFEAFF02
:101BA000EE52E9CF4AF0EACF4BF0DF504A24E96E1B
:101BB000000E4B20EA6EE552E750EF6EBED0020EEB
:101BC000DBCFE9FF030EDBCFEAFFEE52E9CF4AF0AD
:101BD000EACF4BF0DF504A24E96E000E4B20EA6E4C
:101BE000DE0EEF6E020EDBCFE9FF030EDBCFEAFF66
:101BF000EE52E9CF4BF0EACF4CF0DF50DF2A4B2416
:101C0000E96E000E4C20EA6EEFCF4AF0020EDBCFF9
:101C1000E9FF030EDBCFEAFFEE52050EE926000EC8
:101C2000EA22EF504A18E66E020EDBCFE9FF030E00
:101C3000DBCFEAFFEE52050EE926000EEA22E5525E
:101C4000E750EF6EE0C2E9FFE1C2EAFF090EEB5098
:101C5000E66E020EDBCFE9FF030EDBCFEAFFEE52AA
:101C6000E9CF4AF0EACF4BF0DF504A24E96E000E8C
:101C70004B20EA6EE552E750EF6E5FD0020EDBCFED
:101C8000E9FF030EDBCFEAFFEE52E9CF4AF0EACFDD
:101C90004BF0DF504A24E96E000E4B20EA6EDF0E57
:101CA000EF6E020EDBCFE9FF030EDBCFEAFFEE5251
:101CB000E9CF4BF0EACF4CF0DF50DF2A4B24E96E3E
:101CC000000E4C20EA6EEFCF4AF0020EDBCFE9FFA8
:101CD000030EDBCFEAFFEE52050EE926000EEA22E4
:101CE000EF504A18E66E020EDBCFE9FF030EDBCFA2
:101CF000EAFFEE52050EE926000EEA22E552E75011
:101D0000EF6EE0C2E9FFE1C2EAFF090EEB50E66EBA
:101D1000020EDBCFE9FF030EDBCFEAFFEE52E9CF85
:101D20004AF0EACF4BF0DF504A24E96E000E4B2018
:101D3000EA6EE552E750EF6E00D0020EDBCFE9FF0E
:101D4000030EDBCFEAFFEE52E9CF4BF0EACF4CF0C7
:101D5000DF50DF2A4B24E96E000E4C20EA6EEFCFF5
:101D60004AF0020EDBCFE9FF030EDBCFEAFFEE52B3
:101D7000050EE926000EEA22EF504A18E66E020E22
:101D8000DBCFE9FF030EDBCFEAFFEE52050EE926BB
:101D9000000EEA22E552E750EF6E020EDBCFE9FFBC
:101DA000030EDBCFEAFF070EE926000EEA22020E41
:101DB000EF6E020EDBCFE9FF030EDBCFEAFFEE5240
:101DC000050EE926000EEA22EF50E66E020EDBCF8A
:101DD000E9FF030EDBCFEAFFEE52E9CF4AF0EACF8C
:101DE0004BF0DF50DF2A4A24E96E000E4B20EA6EEA
:101DF000E552E750EF6EDF504A6E020EDBCFE9FF8F
:101E0000030EDBCFEAFF4A50070BF36EF80EEF1418
:101E1000F310EF6E020EDBCFE9FF030EDBCFEAFF1C
:101E2000EF8E2E280F0B2E6E01D0148400D0040EDE
:101E3000E15C02E2E16AE552E16EE552E7CFD9FFEB
:101E40001200E0C2E9FFE1C2EAFF070EEB50080D05
:101E5000F3CFE9FFF4CFEAFF000EE926010EEA22F4
:101E6000EF50800B01E188D0E10E426EE0C2E9FF45
:101E7000E1C2EAFF070EEB50436EE0C2E9FFE1C2A8
:101E8000EAFF070EEB50080DF3CFE9FFF4CFEAFFAE
:101E9000000EE926010EEA22EE52EE52EF50446E99
:101EA000E0C2E9FFE1C2EAFF070EEB50080DF3CFF5
:101EB000E9FFF4CFEAFF000EE926010EEA22EE5216
:101EC000EF50456EE0C2E9FFE1C2EAFF070EEB50BA
:101ED000080DF3CFE9FFF4CFEAFF000EE926010E6B
:101EE000EA22030EE926000EEA22EF50466EE0C217
:101EF000E9FFE1C2EAFF070EEB50080DF3CFE9FF5F
:101F0000F4CFEAFF000EE926010EEA22040EE926CC
:101F1000000EEA22EF50476EE0C2E9FFE1C2EAFF9D
:101F2000070EEB50080DF3CFE9FFF4CFEAFF000EE8
:101F3000E926010EEA22050EE926000EEA22EF50FC
:101F4000486EE0C2E9FFE1C2EAFF070EEB50080D60
:101F5000F3CFE9FFF4CFEAFF000EE926010EEA22F3
:101F6000060EE926000EEA22EF50496E080EE66ED4
:101F7000E8EC1AF0E55211D0630E426EE0C2E9FFC0
:101F8000E1C2EAFF070EEB50436E446A030E456E52
:101F9000040EE66EE8EC1AF0E55212001F0E4A6ECF
:101FA000E0C2E9FFE1C2EAFF070EE926000EEA22DD
:101FB0004A50EF16E0C2E9FFE1C2EAFF070EEB501C
:101FC000080DF3CFE9FFF4CFEAFF000EE926010E7A
:101FD000EA22EF9EE0C2E9FFE1C2EAFF070EEB5002
:101FE000080DF3CFE9FFF4CFEAFF000EE926010E5A
:101FF000EA22EE52EE6AED6AE0C2E9FFE1C2EAFFD0
:10200000070EEB50080DF3CFE9FFF4CFEAFF000E07
:10201000E926010EEA22030EE926000EEA22800ECE
:10202000EF6EE0C2E9FFE1C2EAFF070EEB50080DD8
:10203000F3CFE9FFF4CFEAFF000EE926010EEA2212
:10204000040EE926000EEA22EF6AE0C2E9FFE1C2CF
:10205000EAFF070EEB50080DF3CFE9FFF4CFEAFFDC
:10206000000EE926010EEA22050EE926000EEA22FC
:10207000EF6AE0C2E9FFE1C2EAFF070EEB50080D8C
:10208000F3CFE9FFF4CFEAFF000EE926010EEA22C2
:10209000060EE926000EEA22EF6AE0C2E9FFE1C27D
:1020A000EAFF070EEB50080DF3CFE9FFF4CFEAFF8C
:1020B000000EE926010EEA22070EE926000EEA22AA
:1020C000EF6A1200E0C2E9FFE1C2EAFF070EEB503F
:1020D000080DF3CFE9FFF4CFEAFF000EE926010E69
:1020E000EA22070EE926000EEA22050EEF6E120024
:1020F000D9CFE6FFE1CFD9FF020EE1262E50080D21
:10210000F3CF4AF0F4CF4BF0600E4A26020E4B227A
:102110004AC0DEFF4BC0DDFFDECFE9FFDDCFEAFFC7
:10212000EF50800B01E0B1D0E0C2E9FFE1C2EAFF6D
:10213000060EEB50800A40E0200A2BE0600A16E011
:10214000200A01E082D0E0C2E9FFE1C2EAFF0D0E01
:10215000EB50E66EDECFE9FFDDCFEAFFEE52050E73
:10216000E926000EEA22E552E750EF6EE0C2E9FFF1
:10217000E1C2EAFF0C0EEB50E66EDECFE9FFDDCFE9
:10218000EAFFEE52040EE926000EEA22E552E7507D
:10219000EF6EE0C2E9FFE1C2EAFF0B0EEB50E66E24
:1021A000DECFE9FFDDCFEAFFEE52030EE926000E97
:1021B000EA22E552E750EF6EE0C2E9FFE1C2EAFF32
:1021C0000A0EEB50E66EDECFE9FFDDCFEAFFEE52FE
:1021D000020EE926000EEA22E552E750EF6EE0C259
:1021E000E9FFE1C2EAFF090EEB50E66EDECFE9FF40
:1021F000DDCFEAFFEE52010EE926000EEA22E5529B
:10220000E750EF6EE0C2E9FFE1C2EAFF080EEB50D3
:10221000E66EDECFE9FFDDCFEAFFEE52E552E75092
:10222000EF6EE0C2E9FFE1C2EAFF070EEB50070BD9
:10223000E66EDECFE9FFDDCFEAFF070EE926000EEE
:10224000EA22E552E750EF6E00D0E0C2E9FFE1C2BA
:10225000EAFF060EEB50700BE00BE838E840FF0F8A
:102260004A6EDECFE9FFDDCFEAFF4A50070BF36E7F
:10227000F80EEF14F310EF6EDECFE9FFDDCFEAFFCB
:10228000EF8E2E280F0B2E6E01D01484020EE15C0F
:1022900002E2E16AE552E16EE552E7CFD9FF1200B2
:1022A000D9CFE6FFE1CFD9FFE652DF6A200EDF5C2F
:1022B00025E2DF50080DF3CFE9FFF4CFEAFF000E6F
:1022C000E926010EEA22030EE926000EEA22EF506B
:1022D000800B0109E66EDF50080DF3CFE9FFF4CF64
:1022E000EAFF000EE926010EEA22030EE926000E9F
:1022F000EA22E552E750EF6EDF2AD8D7E552E552E1
:10230000E7CFD9FF1200120E326E336AE0C2E9FF46
:10231000E1C2EAFF080EEB50376E8FEF11F0D9CF14
:10232000E6FFE1CFD9FF030EE126DF6A2E50080D4C
:10233000F3CF4AF0F4CF4BF0600E4A26020E4B2248
:10234000010E4AC0DBFF020E4BC0DBFF010EDBCFEC
:10235000E9FF020EDBCFEAFFEF50800B01E059D21C
:10236000010EDBCFE9FF020EDBCFEAFFEE52050ED6
:10237000E926000EEA22EF6AE0C2E9FFE1C2EAFFC5
:10238000070EEB50080DF3CFE9FFF4CFEAFF000E84
:10239000E926010EEA22EE52EE52EF50800B01E1E7
:1023A000A1D0E0C2E9FFE1C2EAFF070EEB50080D41
:1023B000F3CFE9FFF4CFEAFF000EE926010EEA228F
:1023C000EE52EE52EF50E66E010EDBCFE9FF020E49
:1023D000DBCFEAFFEE52E9CF4AF0EACF4BF0DF5015
:1023E0000F014A24E96E000E4B20EA6EE552E750D9
:1023F000EF6E010EDBCFE9FF020EDBCFEAFFEE52FC
:10240000E9CF4AF0EACF4BF0DF50DF2A4A24E96EE9
:10241000000E4B20EA6EEF50E66E010EDBCFE9FFB7
:10242000020EDBCFEAFFEE52050EE926000EEA228D
:10243000E552E750EF6EE0C2E9FFE1C2EAFF070EA6
:10244000EB50080DF3CFE9FFF4CFEAFF000EE926C9
:10245000010EEA22EE52EF50E66E010EDBCFE9FFED
:10246000020EDBCFEAFFEE52E9CF4AF0EACF4BF0A3
:10247000DF504A24E96E000E4B20EA6EE552E75029
:10248000EF6E010EDBCFE9FF020EDBCFEAFFEE526B
:10249000E9CF4BF0EACF4CF0DF50DF2A4B24E96E56
:1024A000000E4C20EA6EEFCF4AF0010EDBCFE9FFC1
:1024B000020EDBCFEAFFEE52050EE926000EEA22FD
:1024C000EF504A18E66E010EDBCFE9FF020EDBCFBC
:1024D000EAFFEE52050EE926000EEA22E552E75029
:1024E000EF6E49D0E0C2E9FFE1C2EAFF070EEB5010
:1024F000080DF3CFE9FFF4CFEAFF000EE926010E45
:10250000EA22EE52EF50E66E010EDBCFE9FF020E3B
:10251000DBCFEAFFEE52E9CF4AF0EACF4BF0DF50D3
:102520000F014A24E96E000E4B20EA6EE552E75097
:10253000EF6E010EDBCFE9FF020EDBCFEAFFEE52BA
:10254000E9CF4AF0EACF4BF0DF50DF2A4A24E96EA8
:10255000000E4B20EA6EEF50E66E010EDBCFE9FF76
:10256000020EDBCFEAFFEE52050EE926000EEA224C
:10257000E552E750EF6EE0C2E9FFE1C2EAFF060E66
:10258000EB50820808E0E0C2E9FFE1C2EAFF060E74
:10259000EB5045081FE133C04CF04D6A030E4C165A
:1025A000000E4D16EC0E4C12000E4D12010EDBCF3C
:1025B000E9FF020EDBCFEAFFEE52E9CF4AF0EACFA5
:1025C0004BF0DF504A24E96E000E4B20EA6E4CC0FF
:1025D000EFFF1ED033C04CF04D6A030E4C16000EB8
:1025E0004D16E80E4C12000E4D12010EDBCFE9FF26
:1025F000020EDBCFEAFFEE52E9CF4AF0EACF4BF012
:10260000DF504A24E96E000E4B20EA6E4CC0EFFF0B
:10261000010EDBCFE9FF020EDBCFEAFFEE52E9CF7E
:102620004BF0EACF4CF0DF50DF2A4B24E96E000E6E
:102630004C20EA6EEFCF4AF0010EDBCFE9FF020E2D
:10264000DBCFEAFFEE52050EE926000EEA22EF503C
:102650004A18E66E010EDBCFE9FF020EDBCFEAFF80
:10266000EE52050EE926000EEA22E552E750EF6E23
:102670003250E66E010EDBCFE9FF020EDBCFEAFF40
:10268000EE52E9CF4AF0EACF4BF0DF504A24E96E30
:10269000000E4B20EA6EE552E750EF6E010EDBCFE5
:1026A000E9FF020EDBCFEAFFEE52E9CF4BF0EACFB3
:1026B0004CF0DF50DF2A4B24E96E000E4C20EA6E0E
:1026C000EFCF4AF0010EDBCFE9FF020EDBCFEAFFCE
:1026D000EE52050EE926000EEA22EF504A18E66E89
:1026E000010EDBCFE9FF020EDBCFEAFFEE52050E53
:1026F000E926000EEA22E552E750EF6E010EDBCF2D
:10270000E9FF020EDBCFEAFFEE52E9CF4AF0EACF53
:102710004BF0DF504A24E96E000E4B20EA6E37C0C2
:10272000EFFF010EDBCFE9FF020EDBCFEAFFEE5237
:10273000E9CF4BF0EACF4CF0DF50DF2A4B24E96EB3
:10274000000E4C20EA6EEFCF4AF0010EDBCFE9FF1E
:10275000020EDBCFEAFFEE52050EE926000EEA225A
:10276000EF504A18E66E010EDBCFE9FF020EDBCF19
:10277000EAFFEE52050EE926000EEA22E552E75086
:10278000EF6E010EDBCFE9FF020EDBCFEAFFEE5268
:10279000050EE926000EEA22EF50E66E010EDBCFB1
:1027A000E9FF020EDBCFEAFFEE52E9CF4AF0EACFB3
:1027B0004BF0DF50DF2A4A24E96E000E4B20EA6E10
:1027C000E552E750EF6EDF504A6E010EDBCFE9FFB6
:1027D000020EDBCFEAFF4A50070BF36EF80EEF1440
:1027E000F310EF6E010EDBCFE9FF020EDBCFEAFF45
:1027F000070EE926000EEA22020EEF6E010EDBCF75
:10280000E9FF020EDBCFEAFFEF8E2E280F0B2E6EB4
:1028100001D01484030EE15C02E2E16AE552E16E4C
:10282000E552E7CFD9FF1200D9CFE6FFE1CFD9FFBC
:10283000E6522F50080DF3CFE9FFF4CFEAFF600E08
:10284000E926020EEA22EF50070B0C6E010E2B6EEA
:10285000DF6A0C50DF5C23E22F50080DF3CFE9FF55
:10286000F4CFEAFF600EE926020EEA22EE52E9CF2B
:102870004AF0EACF4BF0DF500F014A24E96E000E18
:102880004B20EA6EEF50E66EDF50EA6A250FE96EE4
:10289000000EEA22E552E750EF6EDF2ADAD72F501A
:1028A000080DF3CFE9FFF4CFEAFF600EE926020E30
:1028B000EA22070EE926000EEA22EF50010824E280
:1028C0002F50080DF3CFE9FFF4CFEAFF600EE926A1
:1028D000020EEA22070EE926000EEA22EF04E66E57
:1028E0002F50080DF3CFE9FFF4CFEAFF600EE92681
:1028F000020EEA22070EE926000EEA22E552E75010
:10290000EF6E010E306E0ED02F50080DF3CFE9FFA1
:10291000F4CFEAFF600EE926020EEA22EF9E2F288E
:102920000F0B2F6E1390E552E552E7CFD9FF12003F
:10293000D9CFE6FFE1CFD9FF020EE1262C50080DDA
:10294000F3CFE9FFF4CFEAFF000EE926010EEA22F9
:10295000EF50800B01E152D1DF6A2C50080DF3CF0C
:10296000E9FFF4CFEAFF000EE926010EEA22EE525B
:10297000EE52EF50800B41E02C50080DF3CFE9FFF1
:10298000F4CFEAFF000EE926010EEA22EE52EE52E3
:10299000EF50E66EDF50EA6A250FE96E000EEA227C
:1029A000E552E750EF6EDF50DF2AEA6A250FE96E45
:1029B000000EEA22EF502A6E2C50080DF3CFE9FFEB
:1029C000F4CFEAFF000EE926010EEA22EE52EF50A4
:1029D000E66EDF50EA6A250FE96E000EEA22E55244
:1029E000E750EF6EDF50DF2AEA6A250FE96E000E2E
:1029F000EA22EF502A182A6E1FD02C50080DF3CF70
:102A0000E9FFF4CFEAFF000EE926010EEA22EE52BA
:102A1000EF50E66EDF50EA6A250FE96E000EEA22FB
:102A2000E552E750EF6EDF50DF2AEA6A250FE96EC4
:102A3000000EEA22EF502A6E2D50020A66E0030AC9
:102A400049E0010A2CE02C50080DF3CFE9FFF4CF48
:102A5000EAFF000EE926010EEA22030EE926000E27
:102A6000EA22010EEFCFDBFF2C50080DF3CFE9FF78
:102A7000F4CFEAFF000EE926010EEA22EF50600BC8
:102A8000E842E842E842E842E842010A01E188D02F
:102A9000020A72E0010A70E0020A52E095D02C505E
:102AA000080DF3CFE9FFF4CFEAFF000EE926010E8F
:102AB000EA22040EE926000EEA22EF508009E66EB3
:102AC000DF50EA6A250FE96E000EEA22E552E75070
:102AD000EF6E7BD02C50080DF3CFE9FFF4CFEAFF67
:102AE000000EE926010EEA22050EE926000EEA2272
:102AF000EF50B009E66EDF50EA6A250FE96E000E6E
:102B0000EA22E552E750EF6E60D02C50080DF3CF6B
:102B1000E9FFF4CFEAFF000EE926010EEA22060ED5
:102B2000E926000EEA22EF50A009E66EDF50EA6ABD
:102B3000250FE96E000EEA22E552E750EF6E45D010
:102B4000DF50EA6A250FE96E000EEA223F0EEF6EB3
:102B5000DF50DF2AEA6A250FE96E000EEA22EF5005
:102B60002A182A6EDF50EA6A250FE96E000EEA2263
:102B7000010EDBCFEFFF28D0010EDBCFE6FFA5EC87
:102B800008F0E552E76E010EE7CFDBFFDF50EA6A9F
:102B9000250FE96E000EEA22010EDBCFEFFF14D005
:102BA000010EDBCFE6FFD1EC08F0E552E76E010E37
:102BB000E7CFDBFFDF50EA6A250FE96E000EEA225D
:102BC000010EDBCFEFFF00D000D0DF50DF2AEA6A32
:102BD000250FE96E000EEA22EF502A182A6EDF5008
:102BE000DF2AEA6A250FE96E000EEA222AC0EFFF0B
:102BF000DF500C6E010E2B6E139001D02BD8200EDF
:102C0000DF6EDF5000081CE22C2A200E2C5C08E34B
:102C10002C6A010E306E2D2A2D50060801E22D6A15
:102C2000DF062C50080DF3CFE9FFF4CFEAFF000ECA
:102C3000E926010EEA22EF50800B01E0DF6AE1D7BE
:102C4000020EE15C02E2E16AE552E16EE552E7CF95
:102C5000D9FF12002568266A2768030E0C6E010E44
:102C60002B6E1390306A1200020EE66EC5EC19F05E
:102C7000E552146E030EE66EC5EC19F0E552176EC0
:102C800012001750E66E030EE66ED5EC19F0E55211
:102C9000E5521450E66E020EE66ED5EC19F0E552E0
:102CA000E5525D0EE66EE66AD5EC19F0E552E552A6
:102CB0001200E0C2E9FFE1C2EAFF060EEB5008088D
:102CC00004E11594040E426E03D01584050E426E85
:102CD000010EE66EE8EC1AF0E5521200196A158052
:102CE0001298129C129A12960E0EE66E18D8E552A1
:102CF00062C019F01950180803E21590128806D026
:102D0000128C128A150EE66E0AD8E552120012963F
:102D100013880A0EE66E03D8E55215901200D9CF3B
:102D2000E6FFE1CFD9FF12A0FED7000E206E1F6E86
:102D30001E6EFE0EDB50246E030E0B6E140E086E1C
:102D40001290E552E7CFD9FF1200D9CFE6FFE1CFCD
:102D5000D9FF12A0FED720681E681F6AFE0EDB5046
:102D6000246E030E0B6E140E086E1290E552E7CF20
:102D7000D9FF1200E0C2E9FFE1C2EAFF080EEB5002
:102D80004A6E4AC04BF04A6AE0C2E9FFE1C2EAFF7C
:102D9000090EEB5000014A10326E4BC033F0320680
:102DA000000E335AE0C2E9FFE1C2EAFF0B0EEB501E
:102DB000376EE0C2E9FFE1C2EAFF060EEB5082087F
:102DC00008E0E0C2E9FFE1C2EAFF060EEB5083082B
:102DD0000AE1E0C2E9FFE1C2EAFF0A0EEB50376EFA
:102DE0008FEC11F03FD0E0C2E9FFE1C2EAFF070E2D
:102DF000EB50316E87EC16F0E0C2E9FFE1C2EAFF6A
:102E00000A0EEB50366E000E325C040E33581FE291
:102E10001350020B19E11350040B16E1E0C2E9FF55
:102E2000E1C2EAFF060EEB50840802E1138209D0EA
:102E3000E0C2E9FFE1C2EAFF060EEB50A20801E1A1
:102E4000138422D80FD002D0040E446E02D0050E97
:102E5000446E3150436E4C0E426E030EE66EE8EC4B
:102E60001AF0E5521200030E3214346E32C04AF0EA
:102E700033C04BF0D8904B324A32D8904B324A3262
:102E80004A50356E352A120038500F0A01E1D7D169
:102E9000010A01E1CAD1030A01E1A6D1010A01E157
:102EA0007FD1070A01E172D1030A01E143D10F0A80
:102EB00001E131D1010A01E1FBD0030A01E1E9D0CE
:102EC000010A01E1BED0070A01E1B1D0010A31E0F7
:102ED000030A19E0010A01E0B9D11350020B03E122
:102EE0001350040B10E0196A15801298129C129A64
:102EF0001296139613980E0EE66E8FEC16F0E552AE
:102F0000010E386EA3D162C019F01950180807E2FB
:102F100015901288CCD913921394386A97D1128CD9
:102F2000128A150EE66E8FEC16F0E552020E386E20
:102F30008DD112A805D0BBD913921394386A76D0DC
:102F4000020E365C03E0030E365C16E1030E365CBF
:102F500006E1010E356E070E3214346E01D083DFA8
:102F60003550E66EE66A7D0EE66E71D9E552E552A1
:102F7000E5520B0E386E5AD036042DE113A218D04C
:102F800033C04AF04B6A780E4A103A6EEF0E376E35
:102F90003B6A080E396E3750E66E3250E66E3A5094
:102FA000E66E55D9E552E552E552050E386E12D05F
:102FB00033C04AF04B6A7C0E4A103A6E3750E66EC8
:102FC0003250E66E3A50E66E42D9E552E552E5528D
:102FD0000E0E386E2BD0365029E113A215D033C017
:102FE0004AF04B6A740E4A103A6E376A3750372AE5
:102FF000E66E3250E66E3A50E66E29D9E552E55259
:10300000E5520D0E386E12D033C04AF04B6A7C0E7A
:103010004A103A6E3750E66E3250E66E3A50E66E1F
:1030200016D9E552E552E5520E0E386E0FD11296C2
:1030300013880A0EE66E8FEC16F0E552040E386E19
:1030400005D11398390639500AE1129613880A0EF1
:10305000E66E8FEC16F0E5520F0E386EF7D03B504F
:10306000E8243B6E37063BAE04D0080E3710376EAF
:1030700003D0F70E3714376E3750E66E3250E66ED7
:103080003A50E66EE4D8E552E552E552030E386E4A
:10309000DDD03B50E8243B6E12B63B2A12961388D3
:1030A0000A0EE66E8FEC16F0E552060E386ECED0A4
:1030B000139837063906395013E13B5011E1E70EFA
:1030C000376E080E396E3750E66E3250E66E3A5063
:1030D000E66EBDD8E552E552E552070E386E1AD0BD
:1030E00039500CE13B50376E129613880A0EE66E8B
:1030F0008FEC16F0E5520F0E386E0CD03750E66E9E
:103100003250E66E3A50E66EA2D8E552E552E552EC
:10311000050E386E9BD03B50E8243B6E12A63B2A2E
:10312000129613880A0EE66E8FEC16F0E552080E22
:10313000386E8CD013983706390639500DE13B5064
:103140000BE1376A129613880A0EE66E8FEC16F0C2
:10315000E5520F0E386E19D039500BE113861296D6
:1031600013880A0EE66E8FEC16F0E5520F0E386EDD
:103170000CD03750E66E3250E66E3A50E66E67D8A5
:10318000E552E552E552070E386E60D0129613886C
:103190000A0EE66E8FEC16F0E5520C0E386E56D025
:1031A0001398129613A211D0700E34103A6E376A2B
:1031B0003750372AE66EE66A3A50E66E48D8E5524E
:1031C000E552E5520D0E386E0ED0780E34103A6E80
:1031D0003750E66EE66A3A50E66E39D8E552E55267
:1031E000E5520E0E386E32D0375011E01250080BF7
:1031F0000EE13750372AE66E3250E66E3A50E66EF0
:1032000026D8E552E552E5520D0E386E0DD03750F6
:1032100001E113863706129613880A0EE66E8FECCC
:1032200016F0E5520F0E386E11D0129613880A0E62
:10323000E66E8FEC16F0E5520F0E386E07D013983D
:10324000159035D813921394386A00D01200D9CF54
:10325000E6FFE1CFD9FF1296140E086EFE0EDB508A
:103260001E6EFC0EDBCFE6FFFE0EDB50E552E718CC
:10327000216E030E0B6E365002E036040CE1FD0E9B
:10328000DB501F6EFC0EDB50206EFD0EDB50211854
:10329000216E0B2A05D0FC0EDB501F6E2150206ED4
:1032A000080E246E1290E552E7CFD9FF1200322AA1
:1032B000000E33224C0E426E3150436E13A603D0E3
:1032C000010E446E20D012A803D0020E446E1BD013
:1032D00013A212D0850E426E33C04AF04B6A4A5098
:1032E000446E3250456E3750466E050EE66EE8EC81
:1032F0001AF0E5520DD007D012A603D0030E446E8B
:1033000002D0010E446E030EE66EE8EC1AF0E552B0
:103310001200800E6F6E6EAEFED7B00E776E0D018E
:10332000F86B606A030E706E9E0E716E030E726E05
:10333000200E736E010ED46FD56BD86B0F01186B16
:10334000080E196F1A6B1B6B1C6B1D6F1E6B1F6BAE
:10335000800E016F0D01E06BE16BE26BE36BE46BE0
:10336000E56BE66BE76BF06BF16BF26BF36BFA6B93
:10337000FC6B606A0F01506B0E01206B306B406B71
:10338000506B606B706B6F6A1200D9CFE6FFE1CFB4
:10339000D9FFFE0EDB50A96EA69EA69CA680A85063
:1033A00000D0E552E7CFD9FF1200D9CFE6FFE1CF39
:1033B000D9FFFE0EDB50A96EFD0EDB50A86EA69E57
:1033C000A69CA684F29E550EA76EAA0EA76EA68294
:1033D00000000000F28EA1A8FED7A198A694E552A5
:1033E000E7CFD9FF1200D9CFE6FFE1CFD9FF030E17
:1033F000E126FE0EDB50DF6EDF50DF2AE66EC5DF12
:10340000E552E66ED950010FE96EDACFEAFFE552D8
:10341000E750EE6EED6ADFCFE6FFB7DFE5524C6EA8
:103420004CC04DF04C6A010EDB504C104A6E020E3F
:10343000DB504D104B6E010E4AC0DBFF020E4BC03D
:10344000DBFF010EDBCF4AF0020EDBCF4BF04AC0B0
:10345000F3FF4BC0F4FF030EE15C03E200D0E16A2E
:10346000E552E16EE552E7CFD9FF1200D9CFE6FF72
:10347000E1CFD9FFE652FE0EDB50DF6EFC0EDBCF54
:10348000E6FFDF50DF2AE66E90DFE552E552FC0EE4
:10349000DBCF4AF0FD0EDBCF4BF04BC04AF04B6A5E
:1034A0004A50E66EDFCFE6FF80DFE552E552E55297
:1034B000E552E7CFD9FF1200D9CFE6FFE1CFD9FF20
:1034C000020EE126DF6A0A0EDF5C11E2010EDB6A02
:1034D000DB504A6E4B6A4B3404E24A50F508000E4A
:1034E0004B5403E3010EDB2AF3D7DF2AECD7020E9D
:1034F000E15C02E2E16AE552E16EE552E7CFD9FF15
:103500001200D9CFE6FFE1CFD9FFE652DF6A640EA1
:10351000DF5C03E2D1DFDF2AFAD7E552E552E7CFDD
:10352000D9FF1200070E6F14010A15E0010A0DE021
:10353000020E6F5C070B100DF3500201E06FE16BA0
:10354000200EE0270E0EE1230CD00201600EE06F8A
:103550000F0EE16F06D00201500EE06F0F0EE16F0B
:1035600000D0E0C2E9FFE1C2EAFFEF50800B03E0C8
:10357000000E03D002D0010E00D01200D9CFE6FF1A
:10358000E1CFD9FFFE0EDB50426E030EE66E05D88A
:10359000E552E552E7CFD9FF1200D9CFE6FFE1CFE0
:1035A000D9FF1DC04AF04B6A4A50436E1C50446E0E
:1035B000FE0EDBCFE6FF0CD8E552E552E7CFD9FF90
:1035C0001200030E426E010EE66E02D8E5521200A2
:1035D000D9CFE6FFE1CFD9FFFE0EDB50416E0F0ED3
:1035E0003D16B00E3D120A0E1B6E26D8E552E7CFEF
:1035F000D9FF1200D9CFE6FFE1CFD9FF300E426EDE
:10360000FE0EDB50436E020EE66EE2DFE552E5523F
:10361000E7CFD9FF1200B80E426E2550436E2650F8
:10362000446E2750456E2850466E2950476E060E50
:10363000E66ECEDFE5521200D9CFE6FFE1CFD9FF2B
:10364000040EE1260F0130B7FDD7DF6AD950010F14
:10365000E96EDACFEAFF300EEE6E0F0EED6E030E5E
:10366000DB6A0E0EF36E030EDBCFF4FFF350F45C57
:1036700018E2DF50DF2AEA6A3C0FE96E000EEA2208
:10368000EF50E66E010EDBCFE9FFDB2A020EDBCF47
:10369000EAFF01E3DB2AE552E750EF6E030EDB2A77
:1036A000E0D70F0130B7FDD73087040EE15C02E2AE
:0E36B000E16AE552E16EE552E7CFD9FF120064
:020000040030CA
:0100010006F8
:010002000EEF
:0100030010EC
:01000500807A
:010006008079
:010008000FE8
:01000900C036
:01000A000FE6
:01000B00E014
:01000C000FE4
:01000D0040B2
:0200000400F00A
:040000007F0000007D
:0100FF000000
:00000001FF
